 gles2test1

 Timestamp is 4be8d088 (Tue May 11 12:35:36 2010)

 Preferred load address is 00010000

 Start         Length     Name                   Class
 0001:00000000 00000004H .CRT$XCA                CODE
 0001:00000004 00000004H .CRT$XCZ                CODE
 0001:00000008 00000004H .CRT$XIA                CODE
 0001:0000000c 00000004H .CRT$XIZ                CODE
 0001:00000010 00000004H .CRT$XPA                CODE
 0001:00000014 00000004H .CRT$XPZ                CODE
 0001:00000018 00000004H .CRT$XTA                CODE
 0001:0000001c 00000004H .CRT$XTZ                CODE
 0001:00000020 000006a4H .rdata                  CODE
 0001:000006c4 00000027H .rdata$debug            CODE
 0001:000006ec 000026a0H .text                   CODE
 0001:00002d8c 00000018H .xdata                  CODE
 0001:00002da4 0000003cH .idata$2                CODE
 0001:00002de0 00000014H .idata$3                CODE
 0001:00002df4 00000184H .idata$4                CODE
 0001:00002f78 00000026H .idata$6                CODE
 0001:00002f9e 00000000H .edata                  CODE
 0002:00000000 00000184H .idata$5                DATA
 0002:00000188 00000198H .data                   DATA
 0002:00000320 00000040H .bss                    DATA
 0003:00000000 000000c0H .pdata                  DATA

  Address         Publics by Value              Rva+Base       Lib:Object

 0000:00000000       ___safe_se_handler_count   00000000     <absolute>
 0000:00000000       ___safe_se_handler_table   00000000     <absolute>
 0001:00000000       __xc_a                     00011000     corelib0:crt0init.obj
 0001:00000004       __xc_z                     00011004     corelib0:crt0init.obj
 0001:00000008       __xi_a                     00011008     corelib0:crt0init.obj
 0001:0000000c       __xi_z                     0001100c     corelib0:crt0init.obj
 0001:00000010       __xp_a                     00011010     corelib0:crt0init.obj
 0001:00000014       __xp_z                     00011014     corelib0:crt0init.obj
 0001:00000018       __xt_a                     00011018     corelib0:crt0init.obj
 0001:0000001c       __xt_z                     0001101c     corelib0:crt0init.obj
 0001:0000003c       ??_C@_0CD@JFIHFGKD@?2windows?2glsltest1_fragshaderB?4t@ 0001103c     gles2test1.obj
 0001:00000060       ??_C@_0CD@BDBDCEAN@?2windows?2glsltest1_fragshaderA?4t@ 00011060     gles2test1.obj
 0001:00000084       ??_C@_0CC@HPPKLPE@?2windows?2glsltest1_vertshader?4tx@ 00011084     gles2test1.obj
 0001:000000a8       ??_C@_0BA@ECMACICF@EGL_BAD_SURFACE?$AA@ 000110a8     gles2test1.obj
 0001:000000b8       ??_C@_0BC@OMABNJPB@EGL_BAD_PARAMETER?$AA@ 000110b8     gles2test1.obj
 0001:000000cc       ??_C@_0BG@JCAPPMPM@EGL_BAD_NATIVE_WINDOW?$AA@ 000110cc     gles2test1.obj
 0001:000000e4       ??_C@_0BG@IANPFEBH@EGL_BAD_NATIVE_PIXMAP?$AA@ 000110e4     gles2test1.obj
 0001:000000fc       ??_C@_0O@GCFMIHO@EGL_BAD_MATCH?$AA@ 000110fc     gles2test1.obj
 0001:0000010c       ??_C@_0BA@KHKFAGME@EGL_BAD_DISPLAY?$AA@ 0001110c     gles2test1.obj
 0001:0000011c       ??_C@_0BI@KBFIGPCO@EGL_BAD_CURRENT_SURFACE?$AA@ 0001111c     gles2test1.obj
 0001:00000134       ??_C@_0BA@FPCJCEFK@EGL_BAD_CONTEXT?$AA@ 00011134     gles2test1.obj
 0001:00000144       ??_C@_0P@HOPKKPDK@EGL_BAD_CONFIG?$AA@ 00011144     gles2test1.obj
 0001:00000154       ??_C@_0BC@NLAJAPHP@EGL_BAD_ATTRIBUTE?$AA@ 00011154     gles2test1.obj
 0001:00000168       ??_C@_0O@PGDEJDGL@EGL_BAD_ALLOC?$AA@ 00011168     gles2test1.obj
 0001:00000178       ??_C@_0P@ELJNOEME@EGL_BAD_ACCESS?$AA@ 00011178     gles2test1.obj
 0001:00000188       ??_C@_0BE@JIJLFFAN@EGL_NOT_INITIALIZED?$AA@ 00011188     gles2test1.obj
 0001:0000019c       ??_C@_0M@JFIJMCIK@EGL_SUCCESS?$AA@ 0001119c     gles2test1.obj
 0001:000001ec       ??_C@_0CF@GLNKALBC@?8?$CFs?8?5returned?5egl?5error?5?8?$CFs?8?5?$CI0x@ 000111ec     gles2test1.obj
 0001:00000214       ??_C@_0CO@MKHMKJB@Warning?3?5Only?5read?5?$CFu?5bytes?5of?5?$CF@ 00011214     gles2test1.obj
 0001:00000244       ??_C@_0DG@DAFCAJKD@Error?3?5Failed?5to?5allocate?5?$CFd?5byt@ 00011244     gles2test1.obj
 0001:0000027c       ??_C@_0CJ@FEMOKIID@Error?3?5Failed?5to?5open?5shader?5fil@ 0001127c     gles2test1.obj
 0001:000002a8       ??_C@_01KDCPPGHE@r?$AA@    000112a8     gles2test1.obj
 0001:000002ac       ??_C@_0O@OGCHLAPC@inputtexcoord?$AA@ 000112ac     gles2test1.obj
 0001:000002bc       ??_C@_0O@BANECLJM@GL?5ERROR?5?$DN?5?$CFx?$AA@ 000112bc     gles2test1.obj
 0001:000002cc       ??_C@_0CI@GINLBBIE@Error?3?5Failed?5to?5validate?5GLSL?5p@ 000112cc     gles2test1.obj
 0001:000002f4       ??_C@_0CE@JCBAGDPL@Error?3?5Failed?5to?5link?5GLSL?5progr@ 000112f4     gles2test1.obj
 0001:00000318       ??_C@_03GILEGCCJ@mvp?$AA@  00011318     gles2test1.obj
 0001:0000031c       ??_C@_0M@NDDKDOHG@basetexture?$AA@ 0001131c     gles2test1.obj
 0001:00000328       ??_C@_08OAGMDKAF@position?$AA@ 00011328     gles2test1.obj
 0001:00000334       ??_C@_0L@MGILDIMO@inputcolor?$AA@ 00011334     gles2test1.obj
 0001:00000340       ??_C@_0CG@NICEALEG@Error?3?5Failed?5to?5compile?5GLSL?5sh@ 00011340     gles2test1.obj
 0001:00000368       ??_C@_0CH@NPOCEOP@Compiling?5program?5?8?$CFs?8?0?5?$CFd?5bytes@ 00011368     gles2test1.obj
 0001:00000390       ??_C@_0BA@GKADIFMO@eglChooseConfig?$AA@ 00011390     gles2test1.obj
 0001:000003a0       ??_C@_0DG@HMPOADHB@?9?9?9?9?9?9?9?9?9?9?9?9?9?9?9?9?9?9?9?9?9?5finished?5?9@ 000113a0     gles2test1.obj
 0001:000003d8       ??_C@_0P@PNPBPNLI@eglMakeCurrent?$AA@ 000113d8     gles2test1.obj
 0001:000003e8       ??_C@_0BB@KEKMNHDF@eglCreateContext?$AA@ 000113e8     gles2test1.obj
 0001:000003fc       ??_C@_0L@HJOCIPHF@eglBindAPI?$AA@ 000113fc     gles2test1.obj
 0001:00000408       ??_C@_0BH@MDMCFBDG@eglCreateWindowSurface?$AA@ 00011408     gles2test1.obj
 0001:00000420       ??_C@_0O@OMNEJBKO@eglGetConfigs?$AA@ 00011420     gles2test1.obj
 0001:00000430       ??_C@_0O@EEJFKEKH@eglInitialize?$AA@ 00011430     gles2test1.obj
 0001:00000440       ??_C@_0DF@DFKFEDON@?9?9?9?9?9?9?9?9?9?9?9?9?9?9?9?9?9?9?9?9?9?5started?5?9?9@ 00011440     gles2test1.obj
 0001:00000478       ??_C@_1EI@KHNCANBJ@?$AAF?$AAa?$AAi?$AAl?$AAe?$AAd?$AA?5?$AAt?$AAo?$AA?5?$AAc?$AAr?$AAe?$AAa?$AAt?$AAe?$AA?5?$AAt?$AAh?$AAe?$AA?5?$AAd?$AAe?$AAv?$AAi?$AAc?$AAe?$AA?5?$AAc?$AAo?$AAn?$AAt@ 00011478     wince_unittests.obj
 0001:000004c0       ??_C@_1BO@KHIAJBLA@?$AAI?$AAn?$AAi?$AAt?$AAi?$AAa?$AAl?$AAi?$AAz?$AAa?$AAt?$AAi?$AAo?$AAn?$AA?$AA@ 000114c0     wince_unittests.obj
 0001:000004e0       ??_C@_1EI@HEMGLDEE@?$AAF?$AAa?$AAi?$AAl?$AAe?$AAd?$AA?5?$AAt?$AAo?$AA?5?$AAr?$AAe?$AAg?$AAi?$AAs?$AAt?$AAe?$AAr?$AA?5?$AAt?$AAh?$AAe?$AA?5?$AAw?$AAi?$AAn?$AAd?$AAo?$AAw?$AA?5?$AAc?$AAl@ 000114e0     wince_unittests.obj
 0001:00000528       ??_C@_1BM@GPEKOMLI@?$AAP?$AAV?$AAR?$AAS?$AAh?$AAe?$AAl?$AAl?$AAC?$AAl?$AAa?$AAs?$AAs?$AA?$AA@ 00011528     wince_unittests.obj
 0001:00000544       ??_C@_07CHIKDHJG@?9height?$AA@ 00011544     wince_unittests.obj
 0001:0000054c       ??_C@_06EGEBBOP@?9width?$AA@ 0001154c     wince_unittests.obj
 0001:00000554       ??_C@_05MHNCFLJI@?9posy?$AA@ 00011554     wince_unittests.obj
 0001:0000055c       ??_C@_05NOMJGKNJ@?9posx?$AA@ 0001155c     wince_unittests.obj
 0001:00000568       ??_C@_1KE@BDGMONOJ@?$AAH?$AA?3?$AA?2?$AAW?$AAI?$AAN?$AAC?$AAE?$AA6?$AA0?$AA0?$AA?2?$AAP?$AAL?$AAA?$AAT?$AAF?$AAO?$AAR?$AAM?$AA?2?$AAS?$AAM?$AAD?$AAK?$AAV?$AA2?$AA1?$AA0?$AA?2?$AAS?$AAR@ 00011568     wince_unittests.obj
 0001:0000060c       ??_C@_1CI@OHCJFJPM@?$AAE?$AAR?$AAR?$AAO?$AAR?$AA?3?$AA?5?$AA?$CF?$AAs?$AA?5?$AAl?$AAi?$AAn?$AAe?$AA?5?$AA?$CF?$AAd?$AA?3?$AA?5?$AA?$AA@ 0001160c     wince_unittests.obj
 0001:00000634       ??_C@_1CK@MPGKAOE@?$AA?$CI?$AAe?$AAr?$AAr?$AAo?$AAr?$AA?5?$AAc?$AAo?$AAd?$AAe?$AA?3?$AA?5?$AA?$CF?$AAd?$AA?$CJ?$AA?3?$AA?5?$AA?$CF?$AAs?$AA?$AA@ 00011634     wince_unittests.obj
 0001:00000660       ??_C@_1M@DMCDIEDK@?$AAP?$AAK?$AAM?$AA1?$AA?3?$AA?$AA@ 00011660     wince_unittests.obj
 0001:0000066c       ??_C@_0L@GPAGIAIC@?9disablepm?$AA@ 0001166c     wince_unittests.obj
 0001:00000678       ??_C@_1M@ILHOPKA@?$AAE?$AAr?$AAr?$AAo?$AAr?$AA?$AA@ 00011678     wince_unittests.obj
 0001:00000684       ??_C@_1DG@PCJNAHOH@?$AAF?$AAa?$AAi?$AAl?$AAe?$AAd?$AA?5?$AAt?$AAo?$AA?5?$AAg?$AAe?$AAt?$AA?5?$AAm?$AAo?$AAn?$AAi?$AAt?$AAo?$AAr?$AA?5?$AAi?$AAn?$AAf?$AAo?$AA?$AA@ 00011684     wince_unittests.obj
 0001:000006bc       ??_C@_07FBLHGNAH@app?4exe?$AA@ 000116bc     wince_unittests.obj
 0001:00000750       init                       00011750 f   gles2test1.obj
 0001:00000cb4       display                    00011cb4 f   gles2test1.obj
 0001:00000e58       main                       00011e58 f   gles2test1.obj
 0001:000011a8       Normalize                  000121a8 f   maths.obj
 0001:0000136c       myMultMatrix               0001236c f   maths.obj
 0001:000016fc       myPersp                    000126fc f   maths.obj
 0001:000019a0       myTranslate                000129a0 f   maths.obj
 0001:00001c24       myIdentity                 00012c24 f   maths.obj
 0001:00001c6c       myRotate                   00012c6c f   maths.obj
 0001:00002060       AppWndProc                 00013060 f   wince_unittests.obj
 0001:000020c0       WinMain                    000130c0 f   wince_unittests.obj
 0001:000025fc       glGetShaderInfoLog         000135fc f   libGLESv2:libGLESv2.dll
 0001:0000260c       glGetProgramInfoLog        0001360c f   libGLESv2:libGLESv2.dll
 0001:0000261c       glGetAttribLocation        0001361c f   libGLESv2:libGLESv2.dll
 0001:0000262c       glVertexAttribPointer      0001362c f   libGLESv2:libGLESv2.dll
 0001:0000263c       glEnableVertexAttribArray  0001363c f   libGLESv2:libGLESv2.dll
 0001:0000264c       glGetError                 0001364c f   libGLESv2:libGLESv2.dll
 0001:0000265c       glUniform1i                0001365c f   libGLESv2:libGLESv2.dll
 0001:0000266c       glUseProgram               0001366c f   libGLESv2:libGLESv2.dll
 0001:0000267c       glGetUniformLocation       0001367c f   libGLESv2:libGLESv2.dll
 0001:0000268c       glValidateProgram          0001368c f   libGLESv2:libGLESv2.dll
 0001:0000269c       glGetProgramiv             0001369c f   libGLESv2:libGLESv2.dll
 0001:000026ac       glLinkProgram              000136ac f   libGLESv2:libGLESv2.dll
 0001:000026bc       glBindAttribLocation       000136bc f   libGLESv2:libGLESv2.dll
 0001:000026cc       glAttachShader             000136cc f   libGLESv2:libGLESv2.dll
 0001:000026dc       glGetShaderiv              000136dc f   libGLESv2:libGLESv2.dll
 0001:000026ec       glCompileShader            000136ec f   libGLESv2:libGLESv2.dll
 0001:000026fc       glShaderSource             000136fc f   libGLESv2:libGLESv2.dll
 0001:0000270c       glCreateProgram            0001370c f   libGLESv2:libGLESv2.dll
 0001:0000271c       glCreateShader             0001371c f   libGLESv2:libGLESv2.dll
 0001:0000272c       glTexParameterf            0001372c f   libGLESv2:libGLESv2.dll
 0001:0000273c       glTexImage2D               0001373c f   libGLESv2:libGLESv2.dll
 0001:0000274c       glClearColor               0001374c f   libGLESv2:libGLESv2.dll
 0001:0000275c       glDrawArrays               0001375c f   libGLESv2:libGLESv2.dll
 0001:0000276c       glUniformMatrix4fv         0001376c f   libGLESv2:libGLESv2.dll
 0001:0000277c       glDisableVertexAttribArray 0001377c f   libGLESv2:libGLESv2.dll
 0001:0000278c       glClear                    0001378c f   libGLESv2:libGLESv2.dll
 0001:0000279c       GetDC                      0001379c f   coredll:COREDLL.dll
 0001:000027ac       PostQuitMessage            000137ac f   coredll:COREDLL.dll
 0001:000027bc       DefWindowProcW             000137bc f   coredll:COREDLL.dll
 0001:000027cc       ReleasePowerRequirement    000137cc f   coredll:COREDLL.dll
 0001:000027dc       DestroyWindow              000137dc f   coredll:COREDLL.dll
 0001:000027ec       ReleaseDC                  000137ec f   coredll:COREDLL.dll
 0001:000027fc       CreateWindowExW            000137fc f   coredll:COREDLL.dll
 0001:0000280c       RegisterClassW             0001380c f   coredll:COREDLL.dll
 0001:0000281c       GetStockObject             0001381c f   coredll:COREDLL.dll
 0001:0000282c       NKDbgPrintfW               0001382c f   coredll:COREDLL.dll
 0001:0000283c       FormatMessageW             0001383c f   coredll:COREDLL.dll
 0001:0000284c       GetLastError               0001384c f   coredll:COREDLL.dll
 0001:0000285c       SetPowerRequirement        0001385c f   coredll:COREDLL.dll
 0001:0000286c       WideCharToMultiByte        0001386c f   coredll:COREDLL.dll
 0001:0000287c       SetCursorPos               0001387c f   coredll:COREDLL.dll
 0001:0000288c       GetCursorPos               0001388c f   coredll:COREDLL.dll
 0001:0000289c       MessageBoxW                0001389c f   coredll:COREDLL.dll
 0001:000028ac       GetMonitorInfo             000138ac f   coredll:COREDLL.dll
 0001:000028bc       MonitorFromPoint           000138bc f   coredll:COREDLL.dll
 0001:000028cc       GetSystemMetrics           000138cc f   coredll:COREDLL.dll
 0001:0000295c       WinMainCRTStartup          0001395c f   corelib0:pegwmain.obj
 0001:00002a58       exit                       00013a58 f   corelib0:cexit.obj
 0001:00002a70       _exit                      00013a70 f   corelib0:cexit.obj
 0001:00002ab0       __GSHandlerCheckCommon     00013ab0 f   corelib0:gshandler.obj
 0001:00002aec       __GSHandlerCheck           00013aec f   corelib0:gshandler.obj
 0001:00002b10       __security_init_cookie     00013b10 f   corelib0:seccinit.obj
 0001:00002b6c       __security_check_cookie    00013b6c f   corelib0:armsecgs.obj
 0001:00002b80       __gsfailure                00013b80 f   corelib0:armsecgs.obj
 0001:00002bc4       _initterm                  00013bc4 f   corelib0:crt0dat.obj
 0001:00002bf8       _cinit                     00013bf8 f   corelib0:crt0dat.obj
 0001:00002c2c       fprintf                    00013c2c f   corelib1:COREDLL.dll
 0001:00002c3c       _getstdfilex               00013c3c f   corelib1:COREDLL.dll
 0001:00002c4c       fread                      00013c4c f   corelib1:COREDLL.dll
 0001:00002c5c       fclose                     00013c5c f   corelib1:COREDLL.dll
 0001:00002c6c       malloc                     00013c6c f   corelib1:COREDLL.dll
 0001:00002c7c       ftell                      00013c7c f   corelib1:COREDLL.dll
 0001:00002c8c       fseek                      00013c8c f   corelib1:COREDLL.dll
 0001:00002c9c       printf                     00013c9c f   corelib1:COREDLL.dll
 0001:00002cac       fopen                      00013cac f   corelib1:COREDLL.dll
 0001:00002cbc       free                       00013cbc f   corelib1:COREDLL.dll
 0001:00002ccc       sprintf                    00013ccc f   corelib1:COREDLL.dll
 0001:00002cdc       atol                       00013cdc f   corelib1:COREDLL.dll
 0001:00002cec       atoi                       00013cec f   corelib1:COREDLL.dll
 0001:00002cfc       _stricmp                   00013cfc f   corelib1:COREDLL.dll
 0001:00002d0c       _isctype                   00013d0c f   corelib1:COREDLL.dll
 0001:00002d1c       wcslen                     00013d1c f   corelib1:COREDLL.dll
 0001:00002d2c       memset                     00013d2c f   corelib1:COREDLL.dll
 0001:00002d3c       _XcptFilter                00013d3c f   corelib1:COREDLL.dll
 0001:00002d4c       __C_specific_handler       00013d4c f   corelib1:COREDLL.dll
 0001:00002d5c       __security_gen_cookie2     00013d5c f   corelib1:COREDLL.dll
 0001:00002d6c       __report_gsfailure         00013d6c f   corelib1:COREDLL.dll
 0001:00002d7c       TerminateProcess           00013d7c f   coredll:COREDLL.dll
 0001:00002da4       __IMPORT_DESCRIPTOR_libEGL 00013da4     libegl:libEGL.dll
 0001:00002db8       __IMPORT_DESCRIPTOR_libGLESv2 00013db8     libGLESv2:libGLESv2.dll
 0001:00002dcc       __IMPORT_DESCRIPTOR_COREDLL 00013dcc     coredll:COREDLL.dll
 0001:00002de0       __NULL_IMPORT_DESCRIPTOR   00013de0     libegl:libEGL.dll
 0002:00000000       __imp_GetStockObject       00014000     coredll:COREDLL.dll
 0002:00000004       __imp___report_gsfailure   00014004     corelib1:COREDLL.dll
 0002:00000008       __imp___security_gen_cookie2 00014008     corelib1:COREDLL.dll
 0002:0000000c       __imp___C_specific_handler 0001400c     corelib1:COREDLL.dll
 0002:00000010       __imp__XcptFilter          00014010     corelib1:COREDLL.dll
 0002:00000014       __imp_memset               00014014     corelib1:COREDLL.dll
 0002:00000018       __imp_wcslen               00014018     corelib1:COREDLL.dll
 0002:0000001c       __imp__isctype             0001401c     corelib1:COREDLL.dll
 0002:00000020       __imp__stricmp             00014020     corelib1:COREDLL.dll
 0002:00000024       __imp_atoi                 00014024     corelib1:COREDLL.dll
 0002:00000028       __imp___negs               00014028     corelib1:COREDLL.dll
 0002:0000002c       __imp_cos                  0001402c     corelib1:COREDLL.dll
 0002:00000030       __imp_sin                  00014030     corelib1:COREDLL.dll
 0002:00000034       __imp___subs               00014034     corelib1:COREDLL.dll
 0002:00000038       __imp___divs               00014038     corelib1:COREDLL.dll
 0002:0000003c       __imp___dtos               0001403c     corelib1:COREDLL.dll
 0002:00000040       __imp_sqrt                 00014040     corelib1:COREDLL.dll
 0002:00000044       __imp___stod               00014044     corelib1:COREDLL.dll
 0002:00000048       __imp___eqs                00014048     corelib1:COREDLL.dll
 0002:0000004c       __imp___les                0001404c     corelib1:COREDLL.dll
 0002:00000050       __imp___adds               00014050     corelib1:COREDLL.dll
 0002:00000054       __imp_atol                 00014054     corelib1:COREDLL.dll
 0002:00000058       __imp___muls               00014058     corelib1:COREDLL.dll
 0002:0000005c       __imp___itos               0001405c     corelib1:COREDLL.dll
 0002:00000060       __imp_sprintf              00014060     corelib1:COREDLL.dll
 0002:00000064       __imp_free                 00014064     corelib1:COREDLL.dll
 0002:00000068       __imp_fopen                00014068     corelib1:COREDLL.dll
 0002:0000006c       __imp_printf               0001406c     corelib1:COREDLL.dll
 0002:00000070       __imp_fseek                00014070     corelib1:COREDLL.dll
 0002:00000074       __imp_ftell                00014074     corelib1:COREDLL.dll
 0002:00000078       __imp_malloc               00014078     corelib1:COREDLL.dll
 0002:0000007c       __imp_fclose               0001407c     corelib1:COREDLL.dll
 0002:00000080       __imp_fread                00014080     corelib1:COREDLL.dll
 0002:00000084       __imp__getstdfilex         00014084     corelib1:COREDLL.dll
 0002:00000088       __imp_fprintf              00014088     corelib1:COREDLL.dll
 0002:0000008c       __imp_GetSystemMetrics     0001408c     coredll:COREDLL.dll
 0002:00000090       __imp_MonitorFromPoint     00014090     coredll:COREDLL.dll
 0002:00000094       __imp_GetDC                00014094     coredll:COREDLL.dll
 0002:00000098       __imp_PostQuitMessage      00014098     coredll:COREDLL.dll
 0002:0000009c       __imp_DefWindowProcW       0001409c     coredll:COREDLL.dll
 0002:000000a0       __imp_ReleasePowerRequirement 000140a0     coredll:COREDLL.dll
 0002:000000a4       __imp_DestroyWindow        000140a4     coredll:COREDLL.dll
 0002:000000a8       __imp_ReleaseDC            000140a8     coredll:COREDLL.dll
 0002:000000ac       __imp_CreateWindowExW      000140ac     coredll:COREDLL.dll
 0002:000000b0       __imp_RegisterClassW       000140b0     coredll:COREDLL.dll
 0002:000000b4       __imp_TerminateProcess     000140b4     coredll:COREDLL.dll
 0002:000000b8       __imp_NKDbgPrintfW         000140b8     coredll:COREDLL.dll
 0002:000000bc       __imp_FormatMessageW       000140bc     coredll:COREDLL.dll
 0002:000000c0       __imp_GetLastError         000140c0     coredll:COREDLL.dll
 0002:000000c4       __imp_SetPowerRequirement  000140c4     coredll:COREDLL.dll
 0002:000000c8       __imp_WideCharToMultiByte  000140c8     coredll:COREDLL.dll
 0002:000000cc       __imp_SetCursorPos         000140cc     coredll:COREDLL.dll
 0002:000000d0       __imp_GetCursorPos         000140d0     coredll:COREDLL.dll
 0002:000000d4       __imp_MessageBoxW          000140d4     coredll:COREDLL.dll
 0002:000000d8       __imp_GetMonitorInfo       000140d8     coredll:COREDLL.dll
 0002:000000dc       \177COREDLL_NULL_THUNK_DATA 000140dc     coredll:COREDLL.dll
 0002:000000e0       __imp_eglGetError          000140e0     libegl:libEGL.dll
 0002:000000e4       __imp_eglDestroySurface    000140e4     libegl:libEGL.dll
 0002:000000e8       __imp_eglTerminate         000140e8     libegl:libEGL.dll
 0002:000000ec       __imp_eglSwapBuffers       000140ec     libegl:libEGL.dll
 0002:000000f0       __imp_eglMakeCurrent       000140f0     libegl:libEGL.dll
 0002:000000f4       __imp_eglCreateContext     000140f4     libegl:libEGL.dll
 0002:000000f8       __imp_eglBindAPI           000140f8     libegl:libEGL.dll
 0002:000000fc       __imp_eglCreateWindowSurface 000140fc     libegl:libEGL.dll
 0002:00000100       __imp_eglChooseConfig      00014100     libegl:libEGL.dll
 0002:00000104       __imp_eglGetConfigs        00014104     libegl:libEGL.dll
 0002:00000108       __imp_eglGetDisplay        00014108     libegl:libEGL.dll
 0002:0000010c       __imp_eglInitialize        0001410c     libegl:libEGL.dll
 0002:00000110       __imp_eglDestroyContext    00014110     libegl:libEGL.dll
 0002:00000114       \177libEGL_NULL_THUNK_DATA 00014114     libegl:libEGL.dll
 0002:00000118       __imp_glBindAttribLocation 00014118     libGLESv2:libGLESv2.dll
 0002:0000011c       __imp_glLinkProgram        0001411c     libGLESv2:libGLESv2.dll
 0002:00000120       __imp_glGetProgramiv       00014120     libGLESv2:libGLESv2.dll
 0002:00000124       __imp_glValidateProgram    00014124     libGLESv2:libGLESv2.dll
 0002:00000128       __imp_glGetUniformLocation 00014128     libGLESv2:libGLESv2.dll
 0002:0000012c       __imp_glUseProgram         0001412c     libGLESv2:libGLESv2.dll
 0002:00000130       __imp_glAttachShader       00014130     libGLESv2:libGLESv2.dll
 0002:00000134       __imp_glGetError           00014134     libGLESv2:libGLESv2.dll
 0002:00000138       __imp_glEnableVertexAttribArray 00014138     libGLESv2:libGLESv2.dll
 0002:0000013c       __imp_glVertexAttribPointer 0001413c     libGLESv2:libGLESv2.dll
 0002:00000140       __imp_glGetAttribLocation  00014140     libGLESv2:libGLESv2.dll
 0002:00000144       __imp_glGetProgramInfoLog  00014144     libGLESv2:libGLESv2.dll
 0002:00000148       __imp_glGetShaderInfoLog   00014148     libGLESv2:libGLESv2.dll
 0002:0000014c       __imp_glGetShaderiv        0001414c     libGLESv2:libGLESv2.dll
 0002:00000150       __imp_glCompileShader      00014150     libGLESv2:libGLESv2.dll
 0002:00000154       __imp_glShaderSource       00014154     libGLESv2:libGLESv2.dll
 0002:00000158       __imp_glCreateProgram      00014158     libGLESv2:libGLESv2.dll
 0002:0000015c       __imp_glCreateShader       0001415c     libGLESv2:libGLESv2.dll
 0002:00000160       __imp_glTexParameterf      00014160     libGLESv2:libGLESv2.dll
 0002:00000164       __imp_glTexImage2D         00014164     libGLESv2:libGLESv2.dll
 0002:00000168       __imp_glClearColor         00014168     libGLESv2:libGLESv2.dll
 0002:0000016c       __imp_glDrawArrays         0001416c     libGLESv2:libGLESv2.dll
 0002:00000170       __imp_glUniformMatrix4fv   00014170     libGLESv2:libGLESv2.dll
 0002:00000174       __imp_glDisableVertexAttribArray 00014174     libGLESv2:libGLESv2.dll
 0002:00000178       __imp_glClear              00014178     libGLESv2:libGLESv2.dll
 0002:0000017c       __imp_glUniform1i          0001417c     libGLESv2:libGLESv2.dll
 0002:00000180       \177libGLESv2_NULL_THUNK_DATA 00014180     libGLESv2:libGLESv2.dll
 0002:00000188       projection                 00014188     gles2test1.obj
 0002:000001c8       modelview                  000141c8     gles2test1.obj
 0002:00000208       mvp                        00014208     gles2test1.obj
 0002:00000308       gui32WindowWidth           00014308     wince_unittests.obj
 0002:0000030c       gui32WindowHeight          0001430c     wince_unittests.obj
 0002:00000310       gui32PosX                  00014310     wince_unittests.obj
 0002:00000314       gui32PosY                  00014314     wince_unittests.obj
 0002:00000318       __security_cookie          00014318     corelib0:seccinit.obj
 0002:0000031c       __security_cookie_complement 0001431c     corelib0:seccinit.obj
 0002:00000324       gbWindow                   00014324     wince_unittests.obj
 0002:00000328       ghWnd                      00014328     wince_unittests.obj
 0002:0000032c       pfnRegisteredWndProc       0001432c     wince_unittests.obj
 0002:00000330       _exitflag                  00014330     corelib0:cexit.obj
 0002:00000334       gui32DisplayWidth          00014334     <common>
 0002:00000338       gui32DisplayHeight         00014338     <common>
 0002:00000340       mvp_pos                    00014340     <common>
 0002:00000348       attriblocation             00014348     <common>
 0002:00000350       hProgramHandle             00014350     <common>
 0002:00000358       __onexitend                00014358     <common>
 0002:0000035c       __onexitbegin              0001435c     <common>

 entry point at        0001:0000295c

 Static symbols

 0001:000006ec       handle_egl_error           000116ec f   gles2test1.obj
 0001:000028e4       WinMainCRTStartupHelper    000138e4 f   corelib0:pegwmain.obj
 0001:00002990       doexit                     00013990 f   corelib0:cexit.obj
